:04FFF00023001E00CC
:08FFF800000000000000000001
:03000000022F7A52
:0C2F7A0078FFE4F6D8FD75817E022FC1BF
:1036430057502053657175656E63657200302E3770
:0D365300004A756E203137203230303600CD
:02339C008F267A
:10339E00E4F527F528C3E5289526E5279400502364
:1033AE00900000AF82AE83E4FCFD7B107A27F9F823
:1033BE00D312131E4003A380EA0528E52870D60514
:0333CE002780D283
:0133D10022D9
:1034B6007BFF7A3679431236CF1237627F76123720
:1034C600887BFF7A3679501236CF1237627BFF7AC5
:0934D6003679541236CF02376238
:102CFA00123707123745123691E4F524E4F5257D9B
:102D0A0001AF251235067F0112339CE4FDAF25126F
:102D1A0035060525E525C3940340E40524E524C3C7
:102D2A00940540D81237857B017A01799A75360065
:102D3A0075370CE4FFFE1232D890019AE064AB704A
:102D4A0004A3E064CD603912377690019A74ABF02F
:102D5A00A374CDF0A37401F0E4A3F0A3F0A31213BB
:102D6A00AB3D4CCCCDE49001A3F0A304F0E4A3F076
:102D7A007B017A01799AF53675370CFFFE12331A00
:102D8A0090019CE0D39405400374C0F0C390019E67
:102D9A00E0943C90019DE094004006E4F0A3743B6B
:102DAA00F020970B7D017F01123086D2AF80FE9012
:102DBA00019CE0FDE4FF123086D2AF1234B6E4F58E
:102DCA000E1235E1D20EA296920BA297920C1233F2
:102DDA005CE50E60FCE4F50E1214671236A780F16A
:03378500C2162247
:10357600AD07AC062016FDD216EC5401F5F1EDF5BB
:10358600F330AF0320EF0AE5F130E7FBC216AFF2E6
:04359600227F00226E
:04346000AB07AA0606
:103464002016FDD216EA5401F5F1A2AF9200C2AFC4
:103474008DF2EBF5F3A20092AF30AF0320EF07E536
:06348400F130E7FBC21667
:01348A00221F
:04340600AB07AA0660
:10340A002016FDD216EA54014420F5F1A2AF921516
:10341A00C2AF8DF2EBF5F3A21592AF30AF0320EFF6
:08342A0007E5F130E7FBC216D3
:013432002277
:10352C002016FDD21675F131A2AF9200C2AF8FF208
:10353C00E4F5F3A20092AF30AF0320EF07E5F130D2
:04354C00E7FBC216C1
:013550002258
:05377100E4FD02340636
:05377600E4FF02352C08
:0300730002376BE6
:06376B0053F17FC216328B
:0A32D8008E318F328B338A34893532
:1032E200E4F538F539C3E5399537E5389536502791
:1032F200E5322539FFE5313538FE123576AB33AA92
:1033020034A935853982853883EF1211B20539E542
:073312003970D2053880CEAE
:013319002291
:0A331A008E318F328B338A348935EF
:10332400E4F538F539C3E5399537E538953650274E
:10333400E5322539FFE5313538FEAB33AA34A935FA
:10334400853982853883121173FD1234600539E59D
:073354003970D2053880CE6C
:01335B00224F
:10317900256C660025303264253032642E253034C2
:10318900642C25630025303364253032642E2530C4
:1031990034642C256300252E33660025332E3266D0
:1031A90000244750524D422C412C302E30302C4CAB
:1031B9002C253033642C253033642C002C002C3022
:1031C90030302E302C00573A002C523A002C423A1B
:0131D90000F5
:04377B0041012600E2
:0A35BE00E0FF7E007B017A0079AB8C
:1035C800EF7803C333CE33CED8F92420FFE43EFE90
:0935D8007536007537080232D87F
:10366000EF7803C333CE33CED8F92420FFE43EFEF7
:0936700075360075370802331AA3
:1031DA002094028028900125E004F0E0FF90019DF0
:1031EA00E0FCA3E0FDD39FEC940050359001A4E0ED
:1031FA00601E24FE60248000900125EDF078AB7CEF
:10320A00007D017B017A0179277E007F0802113453
:10321A0090019DA3E0900125F022E4900125F08021
:08322A00039001251235BE22BC
:10300600E4F531F532E53225E02457F8E4F608F622
:103016000532E532700205316414453170E7E4F596
:1030260031F53212115AFF600CB42009740129F9E6
:10303600E43AFA80EEEF6043AE02AF010532E532C4
:10304600700205311425E02457F8A60608A60712D3
:10305600115AFF600D642C6009740129F9E43AFAEB
:1030660080EDEF600CE41211A00429F9E43AFA802D
:0F307600028008E5326414453170A8AE31AF32E4
:013085002228
:10255300753AFF753B31753C79753D01753E0175E3
:102563003F47122282E4FBFA79C87842900147E0A0
:10257300FCA3E0FDA3E0FEA3E0FF120C9B120DF40D
:1025830090014FEEF0A3EFF0900147E0FCA3E0FDD4
:10259300A3E0FEA3E0FFC004C005C006C00790018E
:1025A3004FE0FCA3E0FDE4120DBBE4FBFA79C8782D
:1025B30042120B92A804A905AA06AB07D007D006BE
:1025C300D005D004120A9D90014712139F90014732
:1025D300E0FCA3E0FDA3E0FEA3E0FF120DF49001F5
:1025E30051EEF0A3EFF0900147E0FCA3E0FDA3E080
:1025F300FEA3E0FFC004C005C006C007900151E080
:10260300FCA3E0FDE4120DBBA804A905AA06AB07D1
:10261300D007D006D005D004120A9D9001471213AB
:102623009F900147E0FCA3E0FDA3E0FEA3E0FFE4ED
:10263300FBFA79707842120B9290014712139F9024
:102643000151E0FCA3E0FDE4120DBBE4FBFA797059
:102653007842120C9BC004C005C006C00790014F0E
:10266300E0FCA3E0FDE4120DBBD003D002D001D007
:1026730000120AA1C004C005C006C007E4FBFA7932
:10268300617845900147E0FCA3E0FDA3E0FEA3E0F1
:10269300FF120C9BD003D002D001D000120AA190EC
:1026A300014B12139FAB34AA35A93612115AFF649A
:1026B300576004EFB4531790014BE0FCA3E0FDA374
:1026C300E0FEA3E0FF120DA590014B12139F9001B2
:0C26D3004BE0FCA3E0FDA3E0FEA3E0FF51
:0126DF0022D8
:10359A00753AFF753B31753C79753D01753E01758C
:1035AA003F36122282900136E0FCA3E0FDA3E0FE42
:0335BA00A3E0FF8C
:0135BD0022EB
:082ABA008F348E338D328C3114
:102AC200123738120DF4900147EEF0A3EFF0AF3455
:102AD200AE33AD32AC31123738C004C005C006C0C7
:102AE20007900147E0FCA3E0FDE4120DBBA804A996
:102AF20005AA06AB07D007D006D005D004120A9D5E
:102B0200E4FBFA79707842120B9290014D12139FF6
:102B120090014DE0FCA3E0FDA3E0FEA3E0FF120D57
:102B2200F4900149EEF0A3EFF090014DE0FCA3E038
:102B3200FDA3E0FEA3E0FFC004C005C006C00790ED
:102B42000149E0FCA3E0FDE4120DBBA804A905AA1B
:102B520006AB07D007D006D005D004120A9D90011B
:102B62004D12139F7F007E407D1C7C4690014DE0FC
:102B7200F8A3E0F9A3E0FAA3E0FB120B92120DF422
:102B820090014BEEF0A3EFF07538FF753931753ACD
:102B92007D900147E0FEA3E08E3BF53CA3E0FEA35F
:102BA200E08E3DF53EA3E0FEA3E08E3FF540E4FF5C
:102BB200FEFDFCAB34AA33A932A831120D38500401
:102BC2007F5380027F4E8F417B017A0079BC121ABB
:072BD2002B7B017A0079BCA6
:012BD90022D9
:082BDA008F348E338D328C31F3
:102BE200123738120DF4900147EEF0A3EFF0AF3434
:102BF200AE33AD32AC31123738C004C005C006C0A6
:102C020007900147E0FCA3E0FDE4120DBBA804A974
:102C120005AA06AB07D007D006D005D004120A9D3C
:102C2200E4FBFA79707842120B9290014D12139FD5
:102C320090014DE0FCA3E0FDA3E0FEA3E0FF120D36
:102C4200F4900149EEF0A3EFF090014DE0FCA3E017
:102C5200FDA3E0FEA3E0FFC004C005C006C00790CC
:102C62000149E0FCA3E0FDE4120DBBA804A905AAFA
:102C720006AB07D007D006D005D004120A9D9001FA
:102C82004D12139F7F007E407D1C7C4690014DE0DB
:102C9200F8A3E0F9A3E0FAA3E0FB120B92120DF401
:102CA20090014BEEF0A3EFF07538FF753931753AAC
:102CB2008E900147E0FEA3E08E3BF53CA3E0FEA32D
:102CC200E08E3DF53EA3E0FEA3E08E3FF540E4FF3B
:102CD200FEFDFCAB34AA33A932A831120D385004E0
:102CE2007F5780027F458F417B017A0079BC121A9F
:072CF2002B7B017A0079BC85
:012CF90022B8
:10348B007538FF753931753A9FE4FBFA797A7844D0
:10349B00120C9B8F3E8E3D8D3C8C3B7B017A0079D1
:0B34AB00BC121A2B7B017A0079BC22B6
:103604007538FF753931753AA48F3E8E3D8D3C8CEB
:103614003B7B017A0079BC121A2B7B017A0079BCBE
:013624002283
:10335C00C210E49000B7F0900125F01235BEE4FFE6
:10336C00FE7D207C4190019FE0F8A3E0F9A3E0FAF8
:10337C00A3E0FB120B929000B812139FE490011C77
:10338C00F0C211A294B3920FA297B3920C02002632
:10146700A20C309701B3500AA297920C209703124F
:1014770031DA123729EF70030219CE1236258F267B
:101487009001A5E06003200E05AF26123788E526F8
:1014970024F8602C24FE604524E6600C24036003D6
:1014A7000219A8C20E0219A0E4900126F0E0FF0479
:1014B700F074CC2FF582E43400F583E526F080B292
:1014C700900126E0D394004003E014F07F08123423
:1014D700DF7F201234DF7F081234DF8095900126EA
:1014E700E024CCF582E43400F583E4F0200E0ED23C
:1014F7000E7B017A0079CC121E3E0219A07B017A7D
:101507000079CE900133EBF0A3EAF0A3E9F01213D0
:101517004590012F12139F7F437E4D7D527C509043
:10152700012FE0F8A3E0F9A3E0FAA3E0FBC312134D
:101537003460030219A07B017A0079CC123006854A
:101547005C82855B83E064416003021993AA5DA90D
:101557005EC0038B34855F35856036D00312255313
:101567009000A312139FAA61A9627B01C0038B3469
:10157700856335856436D0031225539000A712136F
:101587009FAA67A9687B0112359A90012112139FC0
:101597002010419000B7E004F0E0C3940A50030222
:1015A70019A0D2109000A3E0FCA3E0FDA3E0FEA3E6
:1015B700E0FF90012712139F9000A7E0FCA3E0FD36
:1015C700A3E0FEA3E0FF90012B12139F7F031236C7
:1015D700F50219A09000A7E0FCA3E0FDA3E0FEA39D
:1015E700E0F5358E348D338C32A3E0FCA3E0FDA308
:1015F700E0FEA3E0F5398E388D378C36A3E0FCA3E7
:10160700E0FDA3E0FEA3E0F53D8E3C8D3B8C3A75F3
:101617003E01753F007540B3754101754201754341
:101627001D9000A3E0FCA3E0FDA3E0FEA3E0FF12F2
:101637000076900125E0FFD394004006EF14F52DC6
:1016470080028F2D7538FF753931753AAA753B00C1
:10165700852D3C900125E0753D00F53E7B017A0024
:1016670079CC121A2B9000ABE0FCA3E0FDA3E0FEBF
:10167700A3E0FF122ABA8B318A3289337B017A00C1
:1016870079CC1232327531FF7532317533C57B0132
:101697007A0079CC1232329000AFE0FCA3E0FDA3D0
:1016A700E0FEA3E0FF122BDA8B318A3289337B010C
:1016B7007A0079CC1232327531FF7532317533C504
:1016C7007B017A0079CC1232329000B3E0FCA3E0C0
:1016D700FDA3E0FEA3E0FF12348B8B318A328933FE
:1016E7007B017A0079CC1232327531FF7532317550
:1016F70033C57B017A0079CC12323290011DE0FCB0
:10170700A3E0FDA3E0FEA3E0FF1236048B318A328B
:1017170089337B017A0079CC1232327531FF753209
:10172700317533C77B017A0079CC123232A20F3080
:101737009401B350062094031231DAA294920F75E4
:101747002756E4F5289001A3E0703CE4FFFE7D7A7C
:101757007C4490019FE0F8A3E0F9A3E0FAA3E0FB43
:10176700120B929000B3E0F8A3E0F9A3E0FAA3E02C
:10177700FB120D3840030218407F031236F5752718
:10178700411231DA0218402011030218139000B8F1
:10179700E0FCA3E0FDA3E0FEA3E0FF9000B3E0F8C8
:1017A700A3E0F9A3E0FAA3E0FB120D38600A4008B2
:1017B70090011CE004F08005E490011CF090011CEE
:1017C700E0D3940340307F031236F5752741123179
:1017D700DAE4FFFE7D207C4190019FE0F8A3E0F969
:1017E700A3E0FAA3E0FB120B929000B812139FC27A
:1017F70011E490011CF09000B3E0FCA3E0FDA3E02E
:10180700FEA3E0FF9000B812139F802DE4FFFE7D3A
:101817007A7C4490019FE0F8A3E0F9A3E0FAA3E003
:10182700FB120B929000B3E0F8A3E0F9A3E0FAA350
:10183700E0FB120D385002D2117531007532007578
:1018470033277B017A0079CC123232E4F52CF52A62
:10185700752B017B017A0079CC12000EC3E52B9F13
:10186700EE6480F8E52A648098501974CC252BF52E
:10187700827400352AF583E0622C052BE52B70D3A3
:10188700052A80CF9001A5E070157B017A0079CCFD
:101897001236CF7F2A123788AF2C12367980647BB5
:1018A700FF7A3179CF1236CFE52D04FF1236797FD3
:1018B7002C123788900125E004FF1236797BFF7AD6
:1018C7003179D21236CF9000B3E0FCA3E0FDA3E05C
:1018D700FEA3E0FF120DF47B007A00790012284E78
:1018E7007BFF7A3179D61236CF90011DE0FCA3E059
:1018F700FDA3E0FEA3E0FF120DF47B007A00790060
:1019070012284E123762900121E0F8A3E0F9A3E014
:10191700FAA3E0FB90011DE0FCA3E0FDA3E0FEA31A
:10192700E0FF120A9D120DF48E2A8F2BD3E52B941C
:10193700B4E52A64809480400C7498252BF52B74A9
:10194700FE352AF52AC3E52B944CE52A6480947F5B
:10195700500C7468252BF52B7401352AF52AC3E53D
:101967002B9405E52A6480948050047D01801FD361
:10197700E52B9405E52A648094804004E4FD800209
:101987007D017F011235067D01E48009E4FD7F01B9
:10199700123506E4FDFF123506E4900126F0021425
:1019A70079900126E0FF04F074CC2FF582E434002F
:1019B700F583E526F0900126E0C394505003021406
:0719C70079E014F00214792D
:0119CE0022F6
:10370700E4F5847585FF53912FF592F5A475A5FF10
:01371700228F
:10369100C214E4FDFF123506E4FD7F01123506E494
:0636A100FD7F0202350668
:10350600EF1460101460162402701ABD0103C2A7DE
:1035160022D2A722BD0103C2A622D2A622BD010342
:06352600D28022C28022C7
:1036F500EF24FD700CD214750DFA7D017F02123591
:0237050006229A
:1036A700E50DD39400400CD50D09C214E4FD7F024B
:0436B70012350622A0
:1033D20025640020200053657474696E67733A0097
:1033E20041727269766552616E67653D00206D00BB
:1033F2005365714D6F64653D004379636C654D6F34
:0434020064653D00C0
:061E3E008B2E8A2F893073
:101E4400123551AB2EAA2FA93012115A900136F037
:101E5400121405207E411E8C422015432132441E5B
:101E640089451F564C202D4E21FA5020CA511E85FB
:101E740052216053212F561EC05720F559000022CD
:101E84000343A20822023776AB2EE5302402F9E49C
:101E9400352FFA753AFF753B33753CD2753D0175A4
:101EA4003E01753F45122282900145A3E090019CBA
:101EB400F0D39405400374C0F002206EAB2EE530DD
:101EC4002402F9E4352FFA123006AA57A9587B01E7
:101ED400C003753AFF753B33753CD28B3D753E01AB
:101EE400753F45D003122282AA59A95A7B01C00327
:101EF4008B34855B35855C36D00312255390013BCA
:101F040012139FAA5DA95E7B01C0038B34855F35E4
:101F1400856036D00312255390013F12139F900120
:101F240045E0FEA3E0FFD39400EE64809480500368
:101F3400022203D3EF943CEE648094804003022297
:101F440003EF24FFFFEE34FFFE7B017A01793B02AD
:101F54003660E4900143F0A3F090019DE0FEA3E01D
:101F6400FF900143E0FCA3E0FDC39FEC9E4003020D
:101F74002203C3ED943CEC6480948040030222036A
:101F8400900143E0FEA3E0FF7B017A01793B123527
:101F9400C8900144E02401FF900143E03400FE3383
:101FA40095E0FDFC7B007A00790012284E7BFF7AD5
:101FB4003379D51236CF90013BE0FCA3E0FDA3E0DA
:101FC400FEA3E0FF122ABA900138EBF0A3EAF0A3D3
:101FD400E9F01236CF7BFF7A3379D51236CF9001F0
:101FE4003FE0FCA3E0FDA3E0FEA3E0FF122BDA90A8
:101FF4000138EBF0A3EAF0A3E9F01236CF1237620E
:10200400900144E004F07006900143E004F0021FE4
:102014005D123776E490019DF0A3F07B017A01799B
:102024009AF53675370C02215BAB2EE5302402F9A4
:10203400E4352FFA753AFF753B33753CD2753D0193
:10204400753E01753F45122282900145E0FEA3E0F2
:10205400FF90019DEEF0A3EFF0C3943CEE9400409A
:102064000990019DE4F0A3743BF07B017A01799A15
:1020740075360075370CE402215BAB2EE530240283
:10208400F9E4352FFA753AFF753B33753CD2753D4B
:1020940001753E01753F45122282900145E0FCA383
:1020A400E0FDEC120DBBE4FBFA797A7844120C9B48
:1020B40090019F12139F7B017A01799A75360075FE
:1020C400370CE402215BAB2EAA2FA9309000021238
:1020D4001173B444089001A37401F08005E49001E5
:1020E400A3F07B017A01799A75360075370CE48088
:1020F40066AB2EAA2FA93090000212117324CF6070
:102104000E24DF601180009001A47401F0800DE4BE
:102114009001A4F080069001A47402F07B017A017E
:10212400799A75360075370CE4802C0234B6AB2EE0
:10213400AA2FA930900002121173B431089001A59E
:102144007401F08005E49001A5F07B017A01799A8D
:1021540075360075370CE4FFFE02331A7BFF7A33C1
:1021640079D81236CF1237627BFF7A3379E212368E
:10217400CFE4FFFE7D7A7C4490019FE0F8A3E0F970
:10218400A3E0FAA3E0FB120B92120DF47B007A0099
:10219400790012284E7BFF7A3379EF1236CF12374B
:1021A400627BFF7A3379F21236CF9001A3E0700498
:1021B4007F4180027F441237881237627BFF7A3373
:1021C40079FB1236CF9001A4E0600F24FE60130463
:1021D40070169001377448F0800E9001377431F016
:1021E40080069001377452F0900137E0FF1237886F
:0F21F4001237620237627D017F0112308680FE52
:0122030022B8
:10002600E4F529F528F527F526AB29AA28A927A856
:1000360026AF29AE28AD27AC26120A9DC004C005FE
:10004600C006C007AB29AA28A927A826AF29AE282B
:10005600AD27AC26120A9DD003D002D001D00012E3
:0A0066000C9B8F0B8E0A8D098C088D
:01007000226D
:080076008F318E308D2F8C2E8E
:10007E009001361213AB3B5CA8F190013A1213AB10
:10008E004AC2A72890013E1213AB29612E1390018C
:10009E00421213AB42652EE0900136E0F8A3E0F970
:1000AE00A3E0FAA3E0FBE4FFFE7D807C3F120A9DF5
:1000BE0090014612139F900142E0F8A3E0F9A3E0ED
:1000CE00FAA3E0FBAF31AE30AD2FAC2E120C9B126B
:1000DE002770900146E0F8A3E0F9A3E0FAA3E0FB55
:1000EE00120B9290014A12139F900142E0F8A3E086
:1000FE00F9A3E0FAA3E0FBAF39AE38AD37AC361258
:10010E000C9B122770900146E0F8A3E0F9A3E0FAE9
:10011E00A3E0FB120B9290014E12139F90014AE046
:10012E00FCA3E0FDA3E0FEA3E0FFA804A905AA0638
:10013E00FB120B92E4FBFA7980783F120AA1122E81
:10014E00D4A804A905AA06AB07E4FFFE7D807C3F78
:10015E00120C9B90015212139F90014AE0FCA3E0F7
:10016E00FDA3E0FEA3E0FF900152E0F8A3E0F9A3A7
:10017E00E0FAA3E0FB120B9290015612139F90012E
:10018E004EE0FCA3E0FDA3E0FEA3E0FFA804A9055A
:10019E00AA06FB120B92E4FBFA7980783F120AA1B1
:1001AE00122ED4A804A905AA06AB07E4FFFE7D8093
:1001BE007C3F120C9B90015A12139F90015AE0FC47
:1001CE00A3E0FDA3E0FEA3E0FF900152E0F8A3E060
:1001DE00F9A3E0FAA3E0FB120B9290015E12139FBB
:1001EE0090014EE0FCA3E0FDA3E0FEA3E0FF900132
:1001FE005EE0F8A3E0F9A3E0FAA3E0FB120B929005
:10020E00016212139F90014AE0FCA3E0FDA3E0FE01
:10021E00A3E0FF900162E0F8A3E0F9A3E0FAA3E007
:10022E00FB120B9290016612139FAB35AA34A933C1
:10023E00A832AF3DAE3CAD3BAC3A120A9D900142A6
:10024E00E0F8A3E0F9A3E0FAA3E0FB120C9B900107
:10025E006A12139F90016AE0FCA3E0FDA3E0FEA3E7
:10026E00E0FF12273E90017212139F90016AE0FC8C
:10027E00A3E0FDA3E0FEA3E0FF1227289001761273
:10028E00139F900172E0FCA3E0FDA3E0FEA3E0FF4C
:10029E0090015AE0F8A3E0F9A3E0FAA3E0FB120BF9
:1002AE009290014A12139F90015AE0FCA3E0FDA325
:1002BE00E0FEA3E0FF900156E0F8A3E0F9A3E0FA18
:1002CE00A3E0FB120B92900176E0F8A3E0F9A3E015
:1002DE00FAA3E0FB120B92A804A905AA06AB07909D
:1002EE000162E0FCA3E0FDA3E0FEA3E0FF120A9D85
:1002FE0090014E12139F90014EE0FCA3E0FDA3E08F
:10030E00FEA3E0FFA804A905AA06FB120B92C004E7
:10031E00C005C006C00790014AE0FCA3E0FDA3E0C3
:10032E00FEA3E0FFA804A905AA06FB120B92D003B8
:10033E00D002D001D000120AA1122ED490017A124E
:10034E00139F900176E0FCA3E0FDA3E0FEA3E0FF87
:10035E0090015EE0F8A3E0F9A3E0FAA3E0FB120B34
:10036E0092900166E0F8A3E0F9A3E0FAA3E0FB1295
:10037E000AA190017E12139F90017EE0FCA3E0FD86
:10038E00A3E0FEA3E0F54B8E4A8D498C4890017A8E
:10039E00E0FCA3E0FDA3E0FEA3E0FF123106900116
:1003AE009212139F900172E0FCA3E0FDA3E0FEA366
:1003BE00E0FF90015EE0F8A3E0F9A3E0FAA3E0FB12
:1003CE00120B9290017AE0F8A3E0F9A3E0FAA3E011
:1003DE00FB120C9B90019612139F900196E0FCA3CA
:1003EE00E0FDA3E0FEA3E0FF120DA5900196E0F85C
:1003FE00A3E0F9A3E0FAA3E0FB120B92E4FBFA7977
:10040E0080783F120AA190018612139F900166E038
:10041E00FCA3E0FDA3E0FEA3E0FFA804A905AA0645
:10042E00FB120AA190018212139FE4FFFEFDFC90C5
:10043E000186E0F8A3E0F9A3E0FAA3E0FB120D3881
:10044E00603B4039900182E0FCA3E0FDA3E0FEA3F7
:10045E00E0FF120DA5900186E0F8A3E0F9A3E0FA03
:10046E00A3E0FB120C9B90017EE0F8A3E0F9A3E061
:10047E00FAA3E0FB120AA190018212139F9001824F
:10048E00E0FCA3E0FDA3E0FEA3E0FFA804A905AAFB
:10049E0006FB120B92E4FBFAF97840120B92E4FB86
:1004AE00FA798078BF120AA190018E12139FE4FF91
:1004BE00FE7D407CC0900186E0F8A3E0F9A3E0FA4F
:1004CE00A3E0FB120B92E4FBFA79807840120AA1AA
:1004DE00900136E0F8A3E0F9A3E0FAA3E0FB120BDB
:1004EE0092E4FBFA79807840120AA1900186E0F836
:1004FE00A3E0F9A3E0FAA3E0FB120B92900136E021
:10050E00F8A3E0F9A3E0FAA3E0FB120B92E4FBFAE6
:10051E0079807841120C9B90018A12139F90016A88
:10052E00E0FCA3E0FDA3E0FEA3E0FFA312139F9067
:10053E00017EE0FCA3E0FDA3E0FEA3E0FF90018EB0
:10054E00E0F8A3E0F9A3E0FAA3E0FB120B9290010E
:10055E008AE0F8A3E0F9A3E0FAA3E0FB120B929075
:10056E000182E0F8A3E0F9A3E0FAA3E0FB120AA1EE
:10057E0090017AE0F8A3E0F9A3E0FAA3E0FB120BF6
:10058E009290018AE0F8A3E0F9A3E0FAA3E0FB124F
:10059E000B92900192E0F8A3E0F9A3E0FAA3E0FB3E
:1005AE00120AA1900196E0F8A3E0F9A3E0FAA3E005
:1005BE00FB120B9290016A12139F90018AE0F8A32E
:1005CE00E0F9A3E0FAA3E0FBE4FFFE7D807C3F129E
:1005DE000A9D90016AE0F8A3E0F9A3E0FAA3E0FB1C
:1005EE00120B92900136E0F8A3E0F9A3E0FAA3E033
:1005FE00FB120B92C004C005C006C007AB35AA346F
:10060E00A933A832AF3DAE3CAD3BAC3A120A9D9039
:10061E000142E0F8A3E0F9A3E0FAA3E0FB120C9B81
:10062E00D003D002D001D000120AA190016A121399
:10063E009F90016AE0F8A3E0F9A3E0FAA3E0FBA320
:10064E00E0FCA3E0FDA3E0FEA3E0FF120A9D12373B
:10065E003890013EE0F8A3E0F9A3E0FAA3E0FB1224
:10066E000D38500302026290014EE0FCA3E0FDA3A0
:10067E00E0FEA3E0F54B8E4A8D498C4890014AE08E
:10068E00FCA3E0FDA3E0FEA3E0FF1231069001669D
:10069E0012139F900172E0FCA3E0FDA3E0FEA3E025
:1006AE00FF900152E0F8A3E0F9A3E0FAA3E0FB12F9
:1006BE000B92C004C005C006C00790015AE0FCA30F
:1006CE00E0FDA3E0FEA3E0FF900156E0F8A3E0F901
:1006DE00A3E0FAA3E0FB120B92C004C005C006C053
:1006EE0007900176E0FCA3E0FDA3E0FEA3E0FF90FF
:1006FE000162E0F8A3E0F9A3E0FAA3E0FB120B928B
:10070E00D003D002D001D000120A9D8F4B8E4A8D9D
:10071E00498C48D007D006D005D0041231067BDBB9
:10072E007A0F79497840120AA190016212139F90B4
:10073E000146E0F8A3E0F9A3E0FAA3E0FBE4FFFE34
:10074E007D807C3F120C9B900146E0F8A3E0F9A35C
:10075E00E0FAA3E0FB120C9BE4FBFA798078BF125F
:10076E000AA1900186E0F8A3E0F9A3E0FAA3E0FB6A
:10077E00120B92E4FBFA7980783F120AA1122ED462
:10078E00E4FBFA7980783F120AA190016A12139F56
:10079E00E4FFFEFD7CC090016AE0F8A3E0F9A3E05F
:1007AE00FAA3E0FB120AA190016AE0F8A3E0F9A314
:1007BE00E0FAA3E0FB120C9B90016A12139F9001CA
:1007CE006AE0F8A3E0F9A3E0FAA3E0FBE4FFFE7D04
:1007DE00807C3F120A9D90018A12139F90016AE05D
:1007EE00FCA3E0FDA3E0FEA3E0FF90016AE0F8A306
:1007FE00E0F9A3E0FAA3E0FB120B92E4FBFA798096
:10080E007840120C9BE4FBFA7980783F120AA19093
:10081E00018AE0F8A3E0F9A3E0FAA3E0FB120C9B37
:10082E0090018A12139FE4FFFE7DC07C3E90016A08
:10083E00E0F8A3E0F9A3E0FAA3E0FB120B9290011B
:10084E006AE0F8A3E0F9A3E0FAA3E0FB120B92E44E
:10085E00FBFA798078BF120AA190016AE0F8A3E052
:10086E00F9A3E0FAA3E0FB120B9290016E12139F14
:10087E0090017EE0FCA3E0FDA3E0FEA3E0FF90016B
:10088E008EE0F8A3E0F9A3E0FAA3E0FB120B92903E
:10089E00016A12139F90018EE0FCA3E0FDA3E0FE1F
:1008AE00A3E0FF90018EE0F8A3E0F9A3E0FAA3E045
:1008BE00FB120B92A804A905AA06AB07E4FFFE7D66
:1008CE00807C3F120A9D90015E12139F90017AE088
:1008DE00FCA3E0FDA3E0FEA3E0FFA804A905AA0681
:1008EE00FB120B92E4FBFA79807840120B92E4FB38
:1008FE00FA794078C0120AA190015EE0F8A3E0F9FF
:10090E00A3E0FAA3E0FB120B92900182E0F8A3E0C1
:10091E00F9A3E0FAA3E0FB120B9290016EE0F8A3AC
:10092E00E0F9A3E0FAA3E0FB120B92E4FBFA79C024
:10093E007840120C9B90016AE0F8A3E0F9A3E0FA6C
:10094E00A3E0FB120A9D90016EE0F8A3E0F9A3E08C
:10095E00FAA3E0FB120B92E4FBFA79807840120CBA
:10096E009B900182E0F8A3E0F9A3E0FAA3E0FB126A
:10097E000AA190017AE0F8A3E0F9A3E0FAA3E0FB64
:10098E00120B9290016EE0F8A3E0F9A3E0FAA3E057
:10099E00FB120B92900192E0F8A3E0F9A3E0FAA308
:1009AE00E0FB120AA190018AE0F8A3E0F9A3E0FAB5
:1009BE00A3E0FB120B9290013AE0F8A3E0F9A3E05A
:1009CE00FAA3E0FB120B92900146E0F8A3E0F9A324
:1009DE00E0FAA3E0FB120B9290015E12139F9001BE
:1009EE005EE0FCA3E0FDA3E0FEA3E0FFAB3EAA3F6A
:1009FE00A940121365900142E0FCA3E0FDA3E0FEC6
:100A0E00A3E0FF900166E0F8A3E0F9A3E0FAA3E00B
:100A1E00FB120B92AB41AA42A943121365AB41AA3A
:100A2E0042A943121345E4FBFA79B47843120D3808
:100A3E005022AB41AA42A943C003C002C001121307
:100A4E0045E4FBFA79B47843120A9DD001D002D066
:100A5E0003121365AB41AA42A943121345E4FBFAF4
:100A6E00F9F8120D3860244022AB41AA42A943C0C6
:100A7E0003C002C001121345E4FBFA79B4784312A5
:0B0A8E000AA1D001D002D003121365B2
:010A9900223A
:0A374500E4F5955396BF53A27F22CE
:1035E1005389F0438901538FFE758C70E4F58A533A
:1035F100B8FD53B7FDD2A9D28C53890F438990539B
:033601008FEF2226
:03000B0002375960
:09375900050E758C70758A0032B2
:1036BB000D0A003031323334353637383941424315
:0436CB00444546002C
:103086005387BF75985053877FE4F5BABF01054350
:10309600A240800353A2BFE4F5BDED146015146091
:1030A6001A14601F1460242404702575BEF075BFC1
:1030B6000B802375BEF075BF05801B75BEF075BF0E
:1030C60002801375BE7075BF01800B75BEB080039C
:1030D60075BE30E4F5BF75BD035391FE43920143BF
:1030E60091025392FDC21753B8EF53B7EF43B8108E
:1030F600E49000A1F09000A0F09000A2F0D2AC22E3
:0300230002328A1C
:10328A00C0E0C083C082C0D075D0103098309000A2
:10329A00A1E0C3949F50259000A0E0FF04F07400C1
:1032AA002FF582E43400F583E599F09000A1E0045B
:1032BA00F09000A0E0C394A04002E4F0C2983099D4
:0E32CA0004C299C217D0D0D082D083D0E03297
:080003002017FDD2178F99228E
:103433009000A1E0D394004021A3E0FF04F07400C6
:103443002FF582E43400F583E0FF9000A1E014F04F
:0C345300A3E0C394A04005E4F0227F0039
:01345F00224A
:0337880002000339
:103625007F207E4E9000A1E07010D3EF9400EE94C1
:0D363500004007EF1F70ED1E80EA123433D5
:013642002265
:1036CF0012115AFF600C123788740129F9E43AFA83
:0336DF0080EE2258
:0F3729009000A1E0D3940040037F01227F002293
:10367900AE07EE54F0C4540F9036BE93FF1237884C
:08368900EE540F93FF02378895
:093762007BFF7A3679BB0236CFF9
:1035510012115AFF601EC3648094E1400ED3EF64E0
:103561008094FA5006EF24E01211A0740129F9E4C5
:043571003AFA80DCC6
:013575002233
:0E284E008F348E338D328C318B358A3689373C
:10285C00E4F541EC4D4E4F701EE94A4B70057F304C
:10286C00023788AB35AA36A937AF4105418F82753F
:10287C008300743002298EAE33AD32AC31EC335060
:10288C0036E5374536453570077F2D12378880146D
:10289C00AB35AA36A937AF4105418F8275830074D9
:1028AC002D1211B2AF34AE33AD32AC311213108FD6
:1028BC00348E338D328C31754001753B00753ACABC
:1028CC0075399A75383BE4FFFEFDFCAB3BAA3AA97F
:1028DC0039A838D31213345003022979AF34AE33EC
:1028EC00AD32AC31A83812127E8F3F8E3E8D3D8CAE
:1028FC003CEC4D4E4F7004E5407028E53F2430FF12
:10290C00E5374536453570051237888013AB35AA47
:10291C0036A937AE4105418E82758300EF1211B294
:10292C00E4F540AF3BAE3AAD39AC38AB3FAA3EA96B
:10293C003DA83C1211F3AA06A905A804C3E5349FCF
:10294C00F534E5339AF533E53299F532E53198F5FE
:10295C0031AF3BAE3AAD39AC38E47B0AFAF9F81238
:10296C00127E8F3B8E3A8D398C380228D2E5364553
:10297C003745356010AB35AA36A93785418275834A
:05298C0000E41211B28D
:012991002223
:100A9A00020E60E86480F8E933E83360110460F01C
:100AAA00ED33EC337009E8FCE9FDEAFEEBFF2204C2
:100ABA0060DED3EB9FEA9EE99DE8C2E78CF0C2F7BD
:100ACA0095F0400CE8CCF8E9CDF9EACEFAEBCFFB89
:100ADA00120E2B85D0F05804700320D5B3E80470A9
:100AEA00075002B2D5020E6A92D5EC0460F7E4CC44
:100AFA00C0E0C398F8603B94186008400DD0E0FB52
:100B0A00020E42E4FBFAC9FC8028E830E406E4C994
:100B1A00FBE4CAFCE830E305E4C9CACBFCE85407A5
:100B2A006010F8C3E913F9EA13FAEB13FBEC13FCB0
:100B3A00D8F130F52FC3E49CFCEF9BFFEE9AFEED53
:100B4A0099FDD0E0FBEF4E4D4C701222DB03020EF2
:100B5A0067EC2CFCEF33FFEE33FEED33FDED30E7AF
:100B6A00EB020E42EF2BFFEE3AFEED39FDD0E0FB31
:100B7A0050130BBB0003020E6AED13FDEE13FEEFDA
:080B8A0013FFEC13FC020E4204
:100B9200EC4D6011E8497017ED33EC3304600DE45D
:100BA200FCFFFEFD22E933E8330470F8020E601206
:100BB2000E2B58046009E4CC248150062850090207
:100BC2000E6A284003020E67C0E0EB4A7044B98007
:100BD20006D0E0FB020E56EF4E701CBD8008EBFF04
:100BE200EAFEE9FD80EBE98DF0A4FEE5F0020C7B64
:100BF200E9CDF9EAFEEBFFEF89F0A4FCE5F0CE893E
:100C0200F0A42EFFE435F0CD89F0A42DFEE435F0FA
:100C12008067EF4E7005BD80D780C3EF8BF0A4AC28
:100C2200F0EE8BF0A42CFCE435F0F8EF8AF0A42C63
:100C3200E5F038FCE433CB8DF0A42CFCE5F03BF876
:100C4200EE8AF0A42CFCE5F038F8E433CF89F0A466
:100C52002CFCE5F038CF3400CE89F0A42FFFE5F06C
:100C62003EFEE433C98DF0A42EFEE5F039CD8AF0C4
:100C7200A42FFFE5F03EFEE43DFD33D0E0FB50073C
:100C82000BBB000F020E6AEC2CFCEF33FFEE33FEBF
:060C9200ED33FD020E42ED
:100C9800020E6AEC5D046005E859047003020E60F8
:100CA800120E2B580460F6EC4860F2EC7004FDFE5E
:100CB800FF22C860DB2481C85009C398600250062F
:100CC800020E679850CAF582E9294B4A7005AB8233
:100CD800020E5675F0007C1A7880C3EF9BEE9AEDF1
:100CE80099400DC3EF9BFFEE9AFEED99FDE842F0A7
:100CF800DC23ACF0D0E0FFD0E0FED0E0FDAB8220FA
:100D0800E7101BEB60BAEC2CFCEF33FFEE33FEED83
:100D180033FD020E42E803F830E705C0F075F00035
:100D2800EF2FFFEE33FEED33FD40B830E7C280AA67
:100D380074F8CC6480CCC86480C8F582046043C36E
:100D4800EB9FF5F0EA9E42F0E99D42F0E89C45F001
:100D580060305018E5825FFFE582F42B5582FB5026
:100D6800210ABA001D09B90019088016E5825BFB43
:100D7800E582F42F5582FF50090EBE00050DBD0017
:100D8800010CC3EB9FF5F0EA9E42F0E99D42F0E8C2
:0D0D98009C45F06007CC4820E701B3EC2239
:100DA500ED33EC33600A047003BD8004ECB2E7FC5C
:010DB500221B
:100DB60075F020800E75F010800575F0087D007EB8
:100DC600007F003392D530D503121310EC33401058
:100DD600EF33FFEE33FEED33FDEC33FCD5F0ED22C1
:0E0DE600E5F0247EA2D513CC92E7CDCEFF22FD
:100DF400EDD2E7CD33EC3392D524814006E4FFFEF7
:100E0400FDFC22FCE4CFCECDCC24E0501174FF8055
:100E1400EDC3CC13CCCD13CDCE13CECF13CF0470F2
:070E2400F030D5DE021310CF
:1019CF00E54C2438F8E6054C227835300702783894
:1019DF00E475F0011213E502115A2000EB7F2ED2AD
:1019EF00008018EF540F2490D43440D4FF30040BF0
:1019FF00EF24BFB41A0050032461FFE54D600215B8
:101A0F004D0550E5507002054F30070D7835E475E0
:101A1F00F0011213E5EF0211A00234DF7403D207B5
:101A2F008003E4C207F54C8B358A368937E4F54DD0
:101A3F00F54FF550E54D60077F20121A0A80F575B6
:101A4F004EFFC201C200C202C203C205C206C208D3
:101A5F001219D8FF700D3007057F00121A1BAF50F7
:101A6F00AE4F22B4255FC2D5C2041219D8FF24D0BD
:101A7F00B40A00501A75F00A784D30D50508B6FF34
:101A8F000106C6A426F620D5047002D20380D924FD
:101A9F00CFB41A00EF5004C2E5D204021D08D201E0
:101AAF0080C6D20080C0D20280BCD2D580BAD20507
:101ABF0080B47F20121A0A2002077401B54D00402E
:101ACF00F11219CFFF121A0A021A43D208D2068056
:101ADF00951219CFFB1219CFFA1219CFF94A4B7081
:101AEF000679FF7A1D7BFF20022EE54D602A7E00CE
:101AFF008E8275830012117360060EEE654E70F0C4
:101B0F00C2D5EBC0E0EAC0E0E9C0E0EE121D68D03C
:101B1F00E0F9D0E0FAD0E0FB12115AFF60AAEBC057
:101B2F00E0EAC0E0E9C0E0121A0AD0E02401F9D0DF
:101B3F00E03400FAD0E0FBE54E0460DCD54ED980EE
:101B4F0087D20280A2121D4B60F7E54E700104127E
:101B5F000E75A94E600DE54E600914F54E121DF27B
:101B6F00EF60F3EA30E702F404C3995077EAF42503
:101B7F004E0430E701E404F54E800D121D4B60C199
:101B8F00EA054E254E120E75EA784BF630E701E462
:101B9F00254E04D54E0420050114121D68E4C0E043
:101BAF00121DF2784BE6601320E70714F61219F2B4
:101BBF00802204F6D0E014C0E07F001219F2E54E47
:101BCF0060071219E9154E800B3005031219E9D081
:101BDF00E0021A43D0E00480C5121D4B60A0E54E11
:101BEF0004120E75784BEAF6E54E200502600104EB
:051BFF002404121D6822
:101C040074FF04C0E0121DF21219F2E54E20050221
:101C140060031219E9D0E0B54EE87F451219FC784B
:101C24004BE67F2B30E7047F2DF404C0E0121A0A40
:101C3400D0E075F00A84C0F01219F3D0E01219F361
:101C4400021A43791080027908C206C2088008D2B9
:101C5400D5790A8004790AC2D5E54E047002F54E9E
:101C6400E4FAFDFEFF1219CFFC7B082001131219C0
:101C7400CFFD7B1030000A1219CFFE1219CFFF7B63
:101C840020EC3382D592D55013C3E43000069FFF75
:101C9400E49EFEE42001039DFDE49CFCE4CBF8C239
:101CA40001EC700CCFCECDCCE824F8F870F380179B
:101CB400C3EF33FFEE33FEED33FDEC33FCEB33FBCC
:101CC400994002FB0FD8E9EB300105F8D0E0C44895
:101CD400B201C0E00AEC4D4E4F78207B0070C2EA9E
:101CE400B54E0040BCC0E0121D6AD0F0D0E0200127
:101CF40004C4C0E0C4B201C0F01219F3D0F0D5F0AE
:101D0400EB021A431214051AE0531C47581AB14C3B
:101D14001AAD421C4B4F1C53441C53491AC6431C56
:101D240059551B8A461BE8451B54471E1F501AB5BC
:101D34002D1AB92E1ADC2B1ABD231ADA201E082AF2
:101D44001A754800001AD4E54EB4FF03754E061206
:101D540019CFFC1219CFFD1219CFFE1219CFFF783B
:101D640044020EA4790AA2D5200314300509B9103F
:101D7400020404B9080104A2D5200602500104207B
:101D840002689202B54D005034C0E07F2030031940
:101D94007F30A20272067205500F121DC1C202C228
:101DA40006C205C2087F30800F300503E9C0E01287
:101DB4001A0A300503D0E0F9D0E0B54DCC30051750
:101DC4007F30B9100C121A0A7F583004077F7880CC
:101DD40003B90803121A0A3002057F2D021A0A7F7A
:101DE400202008F87F2B2006F322920280CF7F0068
:101DF400B4070050052444F8E6FF22286E756C6C85
:101E04002900D2011219CF3001F8C201784D30D522
:101E14000108F6021A752D504349581219CF2403AC
:101E2400B405004001E4901E1A931219FB743A128F
:0A1E340019FBD203754D04021C4790
:10220400E54C30030104F82328243AF822783730C7
:102214000302783AE475F0011213E502115A60ECF6
:10222400C5507002154F14C550200304FF023780B7
:10223400783774FFF5F00213F5FF0236E2E54D60DE
:1022440006D54D037F002220030F123718EF6008D4
:102254000550E5507002054F2278371213DC121135
:102264005AFF60E97837E475F0011213E580DE1255
:10227400224BEFC0E012223DD0E040F380A0D20315
:102284008002C2038B378A388939E4F54EF54CF560
:102294004FF550754D00C202C200C201C2041222A1
:1022A40011FF7005AF4E7E0022B42530122211FFBB
:1022B40024D0B40A00500C75F00AC54DA4254DF580
:1022C4004D80E924CFB41A00EF5002C2E502251F65
:1022D400D20180D8D20080D4D20480D0EF12223D23
:1022E4005008122273EF600E80A9EFC0E012224B57
:1022F400D0E06F609EEF607412222280A712224BFE
:10230400EF6069E54D7007054D800312224BEF60C5
:102314001420040E122204E475F0011213E5EF12E6
:1023240011A0D54DE6200404054C054E80BA1222B6
:1023340041EFC0E012223DD0E05004122222E4FF1B
:1023440020040E122204E475F0011213E5EF1211B9
:10235400A0EF70DA200404054C054E808BE54D6037
:1023640002054D122273122241EF70C6300304E4B9
:10237400122222E54E60030222A87EFF7FFF22E59F
:102384004D6002054D122273D206D205122241EF8E
:1023940030060260D7C0E0122222D0E0AC51AD5228
:1023A400AE53AF54122DFD8C518D528E538F545019
:1023B4000712224BC20580D4200410200502054ECA
:0823C4001222041213DC054C87
:1023CC00121365022297D0E0809A7900800A791066
:1023DC00800679088002790AD205E54D6002054D28
:1023EC00E9C0E0122273EF60DD12224BBF2D04D244
:1023FC00028003BF2B09122273EF60CA122241D054
:10240C00E0B40A028033B40802802EBF3027700279
:10241C007408C205C0E0122241D0E0BF78028003EC
:10242C00BF5816054DD54D028007D54D04D20580F9
:10243C000B741080197002740ABF000AEFF8E4FCE8
:10244C00FDFEFF0224D2C0E0EF122222D0E0F9E41C
:10245C00FCFDFEFFE9C0E0ECC0E0EDC0E0EEC0E04A
:10246C00EFC0E0122241EFF8D0E0FFD0E0FED0E068
:10247C00FDD0E0FCD0F0E8604DB461004007B47BC7
:10248C00005002C2E524D0503DFA24F6500724F93E
:10249C005034240AFAEAB5F000502BCFA9F0A42F3F
:1024AC00FF92D5E9C5F0CEA4A2D53EFE92D5E9C5E2
:1024BC00F0CDA4A2D53DFD92D5E9C5F0CCA4A2D512
:1024CC003CFCC205808EE8C0E020042A20050805EB
:1024DC004E3002031213101222041213DC054C208E
:1024EC00000B20010DEE8FF01211D4800912136530
:1024FC008004EF1211A0D0E01222220222972004B5
:10250C00101222041213DC054CE54F8550F0121109
:10251C00D480E812140523615323DA5822D84C22B4
:10252C00D44222B04823DE4F23E24423014323D676
:10253C004923E25523834623834523834722DC2A00
:07254C00250A4E000022E009
:0D373800ED33EC3360065004EC6480FC229D
:102ED000020E6022EDA2E7D2E7F9EC3340F260F394
:102EE000B4FF08ED547F70E8020E6AF82481C2E056
:102EF000C0E0F40428FAC313FCED92E7FD8C448D86
:102F0000458E468F47EEA2E7E9BA7F02C31334002D
:102F10009400FA75F091A4E5F013F494FE8AF0A4FD
:102F200033E5F033248CD313FDE492E7FE7F007C7D
:102F30003F758302ECC0E0F8EDC0E0F9EEC0E0FAC6
:102F4000EFC0E0FBAC44AD45AE46AF47120C9BD0A2
:102F5000E0FBD0E0FAD0E0F9D0E0F8120AA1ED648D
:102F600080FD30E7011CD583CBED33CC33F8D0E0C6
:0A2F7000A2E71328C313CC13FD22BF
:103106008F478E468D458C44AB4BAA4AA949A848A1
:10311600120C9B1229B28F478E468D458C44E5488A
:1031260030E747ECC0E0EDC0E0EEC0E0EFC0E0E421
:10313600FFFEFDFCAB47AA46A945A844120D387B05
:10314600DB600250087A0F7949784080067A0F7959
:103156004978C0D0E0FFD0E0FED0E0FDD0E0FC1220
:103166000AA18F478E468D458C44AF47AE46AD4586
:03317600AC442244
:1026E0003A70FA83BCAAE9E43E81E0F8BF9DE9E6CE
:1026F0003F80000039283C1ABB9969663DA335E349
:10270000BF255DE73FC90FDB418DDBCCC44936EE09
:1027100045C9913FC5B0F83D3F800000C317F5346F
:10272000452FFA73C60AFDDD1227CF04A2E19200FD
:102730001420E0159026E07404120FA780261227BB
:10274000CF30E102B20020E0EB8C448D458E468F05
:10275000479026F47404120FA7A844A945AA46ABD3
:1027600047120B92ED4C6007300004EC6480FC22B1
:102770001227CFC0E08C448D458E468F4790271896
:102780007403120FA7A844A945AA46AB47120B929F
:10279000ECC544FCEDC545FDEEC546FEEFC547FF63
:1027A0009027087403120FA7D082A844A945AA460F
:1027B000AB47E58230E007120C9BB20080A6EFCB5E
:1027C000FFEECAFEEDC9FDECC8FC120C9B8095ED36
:1027D00033EC547FCC33920024605007D0E0D0E03B
:1027E000020E607B837AF97922783E120B92EDF922
:1027F00033ECF83324815011EFFBEEFA120DF41292
:102800000DB6ECB2E7FC120AA1ED33EC33602F24D5
:1028100003F8C313FCED92E7FDE82481E4501FECBC
:10282000F8EDF9EEFAEFFB120DF4EF04C2E0FCF55F
:1028300082120DC0ECB2E7FC120AA1E58203FAEDA8
:0E28400033EC3360071413FCED92E7FDEA223F
:100E2B00E9D2E7C933E833F892D5EDD2E7CD33EC0D
:070E3B0033FC5002B2D52286
:100E4200EC30E7100FBF000C0EBE00080DBD000411
:100E52000BEB6014A2D5EB13FCED92E7FD2274FFBD
:100E6200FCFDFEFF22E480F8A2D574FF13FC7D8016
:030E7200E480EF2A
:100E7500F920E72824F950037907E4F42402FB1844
:100E8500DBFDE624FB5014E9600DE4F618E604F6F4
:0F0E9500B40A08E4F6D9F57401F60A22C2D52290
:100EA400ED33EC3392D5FA602AB4FF33EDC2E77B1D
:100EB400FF60067A0E79C9E4227A0E79D220D5042D
:100EC4007A0E79CD224E614E002B494E46002D49B3
:100ED4004E4600E47A08F608DAFC7B00740722E840
:100EE400C0E0ECC0E0EDC0E0EEC0E0EFC0E0EA75C9
:100EF400F010A4CAABF075F04DA42BFBE435F0FC64
:100F0400EA2410FAEB34C5FBEC34D9FCEDC2E7FF5C
:100F140075F056A4F42411C5F0F434C58FF0A42A56
:100F2400E5F03BE43CF620E714121024D0E0FFD0B7
:100F3400E0FED0E0FDD0E0FC120C9B8014F404121F
:100F44001024D0E0FFD0E0FED0E0FDD0E0FC120B96
:100F540092D0E0F8E6FAEDD2E7CD33EC332482FB0D
:100F6400E4C3CF33CFCE33CECD33CD33DBF37B07E6
:100F740075F00A846004F6081B0AE5F0F6088FF0A1
:100F8400740AA4FFACF08EF0740AA42CFEACF050EA
:100F9400010C8DF0740AA42CFDE435F0F608DBDEB8
:030FA400740722AD
:102DEA00C207C208C209C20AF9E4F555F556FCFD44
:102DFA00FEFFE91006EA20090CB42D04D209D322F9
:102E0A00B42B02D32224D0504794095041240A30CB
:102E1A000A15F88556F0740AA42872E74051C5F0DD
:102E2A00704D85F056D322D208C0E0E4FBFA79202F
:102E3A007841120B92ECF8EDF9EEFAEFFBD0E0FCD8
:102E4A00E4120DC0120AA13007B41555D322240A80
:102E5A00200A20B4FE0720071AD207D32224EB60E7
:102E6A000424E0700EA2099207D20AC209D322C32F
:102E7A00020E60E4300A0BE556300902F404A20798
:102E8A0092093008EA255520D2E5A2E7920A5002B3
:102E9A00F404B4260050D8CCC0E0EDC0E0EEC0E0A7
:102EAA00EFC0E0EC121024D0E0FFD0E0FED0E0FD4D
:102EBA00D0E0FC200A05120B928003120C9B300909
:062ECA0003120DA5C32256
:100FA700C0E0EFFBEEFAEDF9ECF8120B92D0E0F5AA
:100FB700F0EFFBEEFAEDF9ECF812137FA3A3A3A36E
:100FC700E8C0E0E9C0E0EAC0E0EBC0E0C0F0120B27
:100FD7009212138FA3A3A3A3120AA1D0F0D0E0FB10
:0D0FE700D0E0FAD0E0F9D0E0F8D5F0D42247
:10299200BE1249253E4CCCCDBEAAAAAB3F80000058
:1029A2003E7ADBB03EED63383F24BC7D3F490FDB0E
:1029B200ED33ECC2E7CC339200B4FF13ED547F60E9
:1029C20003020E607FDB7E0F7DC97C3F022AADC20F
:1029D20001C3947F401E7007EDD2E794904015EF3B
:1029E200FBEEFAEDF9ECF87F007E007D807C3F1271
:1029F2000C9BD201ED33EC33248430E705E4C0E0D4
:102A0200806D04FAEDD2E754F0C333DAFD54073493
:102A1200002323C0E0CCC0E0F8EDC0E0F9EEC0E056
:102A2200FAEFC0E0FBE4120DC0EC24FEFC8C4C8DEE
:102A32004D8E4E8F4F120B927B007A007980783F39
:102A4200120AA1ECC54CB2E7FCEDC54DFDEEC54E38
:102A5200FEEFC54FFFD0E0FBD0E0FAD0E0F9D0E0C6
:102A6200F8120AA1A84CA94DAA4EAB4F120C9B8C8E
:102A72004C8D4D8E4E8F4F9029927403120FA7A842
:102A82004CA94DAA4EAB4F120B92D0E0600F249E80
:102A9200F582E43429F58312138F120AA130010B57
:102AA2007BDB7A0F79C978BF120AA1ED33EC336070
:082AB20006ECA20092E7FC22F1
:100FF4003F8000004120000042C80000447A000005
:10100400461C400047C35000497424004B18968086
:101014004CBEBC205A0E1BCA6753C21C749DC5AE7D
:10102400FB60065407601C2323121052EB543860F3
:101034000912103E12104D120B92ECF8EDF9EEFA73
:10104400EFCB22EB12104D80F1543803241C900F87
:10105400F4FE93FC0EEE93FD0EEE930ECE93FF2260
:102F8600022CFAE493A3F8E493A34003F68001F23B
:102F960008DFF48029E493A3F85407240CC8C3334C
:102FA600C4540F4420C8834004F456800146F6DF1B
:102FB600E4800B010204081020408090377BE47EF9
:102FC600019360BCA3FF543F30E509541FFEE49310
:102FD600A360010ECF54C025E060A840B8E493A3D7
:102FE600FAE493A3F8E493A3C8C582C8CAC583CA02
:102FF600F0A3C8C582C8CAC583CADFE9DEE780BEBA
:01377F000049
:10106400E709F608DFFA8046E709F208DFFA803E6E
:1010740088828C83E709F0A3DFFA8032E309F6085B
:10108400DFFA8078E309F208DFFA807088828C83C3
:10109400E309F0A3DFFA806489828A83E0A3F60877
:1010A400DFFA805889828A83E0A3F208DFFA804C51
:1010B40080D280FA80C680D4806980F28033801028
:1010C40080A680EA809A80A880DA80E280CA803391
:1010D40089828A83ECFAE493A3C8C582C8CCC58309
:1010E400CCF0A3C8C582C8CCC583CCDFE9DEE780D9
:1010F4000D89828A83E493A3F608DFF9ECFAA9F058
:10110400EDFB2289828A83ECFAE0A3C8C582C8CCAD
:10111400C583CCF0A3C8C582C8CCC583CCDFEADEC6
:10112400E880DB89828A83E493A3F208DFF980CC28
:1011340088F0EF60010E4E60C388F0ED2402B40421
:101144000050B9F582EB2402B4040050AF232345C8
:0611540082239010B47329
:10115A00BB010689828A83E0225002E722BBFE0293
:09116A00E32289828A83E49322C6
:10117300BB010CE58229F582E5833AF583E0225031
:1011830006E92582F8E622BBFE06E92582F8E2227B
:0D119300E58229F582E5833AF583E4932295
:1011A000BB010689828A83F0225002F722BBFE012E
:0211B000F32228
:1011B200F8BB010DE58229F582E5833AF583E8F073
:1011C200225006E92582C8F622BBFE05E92582C81F
:0211D200F22207
:1011D400BB010A89828A83F0E5F0A3F0225006F766
:0F11E40009A7F01922BBFE06F3E5F009F3192263
:1011F300E88FF0A4CC8BF0A42CFCE98EF0A42CFC9B
:101203008AF0EDA42CFCEA8EF0A4CDA8F08BF0A418
:101213002DCC3825F0FDE98FF0A42CCD35F0FCEB77
:101223008EF0A4FEA9F0EB8FF0A4CFC5F02ECD393C
:0F123300FEE43CFCEAA42DCE35F0FDE43CFC22A9
:1012420075F008758200EF2FFFEE33FECD33CDCC63
:1012520033CCC58233C5829BED9AEC99E5829840E6
:101262000CF582EE9BFEED9AFDEC99FC0FD5F0D6C3
:10127200E4CEFBE4CDFAE4CCF9A88222B800C1B9ED
:101282000059BA002DEC8BF084CFCECDFCE5F0CB2B
:10129200F97818EF2FFFEE33FEED33FDEC33FCEB64
:1012A20033FB10D703994004EB99FB0FD8E5E4F91F
:1012B200FA227818EF2FFFEE33FEED33FDEC33FC0C
:1012C200C933C910D7059BE99A4007EC9BFCE99A00
:1012D200F90FD8E0E4C9FAE4CCFB2275F010EF2F45
:1012E200FFEE33FEED33FDCC33CCC833C810D70745
:1012F2009BEC9AE899400AED9BFDEC9AFCE899F880
:0E1302000FD5F0DAE4CDFBE4CCFAE4C8F92212
:0E131000C3E49FFFE49EFEE49DFDE49CFC22EE
:10131E00EB9FF5F0EA9E42F0E99D42F0EC6480C846
:06132E0064809845F022E6
:10133400EB9FF5F0EA9E42F0E99D42F0E89C45F00F
:011344002286
:10134500BB010789828A830214375005E9F8021424
:101355002BBBFE05E9F802144389828A8302137FB9
:10136500BB010789828A8302139F5005E9F802149D
:0A1375004FBBFE05E9F802145B22ED
:10137F00E493FC740193FD740293FE740393FF22B4
:10138F00E493F8740193F9740293FA740393FB22B4
:0C139F00ECF0A3EDF0A3EEF0A3EFF022C1
:1013AB00A8828583F0D083D0821213C21213C2128B
:1013BB0013C21213C2E473E493A3C583C5F0C583B0
:1013CB00C8C582C8F0A3C583C5F0C583C8C582C88C
:0113DB0022EF
:0913DC00E6FB08E6FA08E6F92236
:1013E500FAE6FB0808E6F925F0F618E6CA3AF62209
:1013F500FAE6FB0808E625F0F9F618E63AFAF622C9
:10140500D083D082F8E4937012740193700DA3A376
:1014150093F8740193F5828883E47374029368608A
:06142500EFA3A3A380DF8A
:1034DF00EFB40A07740D1234EA740A309811A899E0
:1034EF00B8130CC2983098FDA899C298B811F6304D
:0734FF0099FDC299F5992225
:1037180010180B12374FBF0D027F0A0234DFAF0FAC
:01372800227E
:053780008F0FD218229A
:1036E200EFC394094005EF940E4003BF2003D3803B
:0336F20001C322EF
:103232008B2E8A2F89308B348A358936AB2E053016
:10324200E530AA2F7002052F14F912115A70ED748D
:10325200FF2530F53074FF352FF52FAB310533E5FF
:1032620033AA327002053214F912115AFFAB2E053D
:1032720030E530AA2F7002052F14F9EF1211A07059
:08328200DAAB34AA35A93622AB
:10000E00E4FFFE12115A600C0FEF70010E09E97039
:05001E00F20A80EF2250
:0C142B00E6FC08E6FD08E6FE08E6FF22ED
:0C143700E0FCA3E0FDA3E0FEA3E0FF2228
:0C144300E2FC08E2FD08E2FE08E2FF22E5
:0C144F00ECF608EDF608EEF608EFF622C9
:0C145B00ECF208EDF208EEF208EFF222CD
:0A374F003098FDAF99C2987E002269
:00000001FF
